:1007AB002564000313010A210004FFFFFFFFFFFF75
:1007BB000A210006FFFFFFFFFFFF0E230005FFFFCF
:1007CB00FFFFFFFF523020100A240005FFFFFFFF41
:1007DB00FFFF0E250005FFFFFFFFFFFF02000000DC
:1007EB000E260005FFFFFFFFFFFF020000000212B5
:0E07FB006D6F6E6579203D006572726F720041
:10084F00024F0203092709310000041100110005AE
:10085F002205300000041A961A220004FFFFFFFF42
:10086F00FFFF000000000000000000000001020375
:02087F0004056E
:0F08B200C2A3C2A48F807F017E001208C1D2A40E
:1008C100E4FDFCC3ED9FEC9E5015E4FBFA0BBB006D
:0F08D100010AEB64644A70F50DBD00010C80E470
:0108E00022F5
:0809F300C2A21208B2C2A42244
:0809FB00D2A21208B2C2A4222C
:060882007B007A007908FA
:100888008B6A8A6B896CAB6AAA6BA96C120455FFD8
:1008980060171209FB7401256CF56CE4356BF56B78
:0A08A8007F017E001208C180DD22EE
:1009A2007F381209F37F801209F37F061209F37F61
:0909B2000C1209F37F010209F3A4
:1009BB001208887F881209F3AB67AA68A969020835
:0109CB0088A3
:0C09DB00EF4E6007EF1F70F81E80F52241
:1009350075CBFC75CA6975CDFC75CC69C2AD75C83A
:1009450004EF1FAC0670011E4C600730CFFDC2CF0F
:0509550080EFC2CA2280
:1008E10075CBDC75CA0075CDDC75CC00C2AD75C8A1
:1008F10004EF1FAC0670011E4C600F20CF08300AB8
:0D090100FAC2CAC2CF22C2CF80E7C2CA220A
:10097F007D08AC051DEC6016EE2EFEC295EF33928E
:10098F0097EF2FFFA296E4334206D29580E4D295DB
:02099F00AF06A1
:0109A1002233
:0E09CC00C2937FAA12097F7FFF12097FD29388
:0109DA0022FA
:0D0664007F647E001209357B007A007978F2
:060671008B648A658966B6
:10067700E4F568F5671209CCBFF0037567FD7F0ADB
:100687007E001209DB0567E567C3946440E7E56709
:1006970064FE600302071CC2937FBB12097F8F674A
:1006A700AB64AA65A966740112049BE4F567AB64A1
:1006B700AA65A966120455FFE567C39F50317FFFFE
:1006C70012097FAB64AA65A966856782758300EF07
:1006D7001204AD85678275830012046E6268120486
:1006E70055D394204005D2937F0122056780BF7FB1
:1006F700FF12097FAB64AA65A966856782758300C7
:10070700EF1204ADD29385678275830012046EB52C
:0707170068037F00227F014F
:01071E0022B8
:080809007BFF8B5D8A5E895FB5
:060811008B648A65896614
:10081700E4F568C2937FCC12097FE4F567AB64AA5D
:1008270065A966120455FEE567C39E501385678266
:1008370075830012046EFF626812097F056780DD09
:07084700AF6812097FD29394
:01084E002287
:0C09E700C2927F327E001208E1D2922200
:1005050078517C007D007BFF7A0779FB7E007F08B0
:1005150012042F78087C007D007BFF7A0879037E22
:10052500007F0612042FE4F560F561F562756378C6
:1005350012095A1209E77FF47E011209351209A240
:100545002094FD8018AB5DAA5EA95F90000112049E
:100555006EFF7879E6B50705780EE660107A0779BB
:10056500C5120809120664780EA60780D8E56164ED
:1005750001456070030206632094FD7F467E0002FC
:10058500060F2094E8E56324F6E56234FFC3648032
:100595009480502312088275600075610180CEAB8E
:1005A5005DAA5EA95F90000112046EFF7879E6B539
:1005B5000705780EE660107A0779EB12080912062E
:1005C50064780EA60780D87FC87E001209357BFFA8
:1005D5007A0779D312080B120664780EA607AB5D6D
:1005E500AA5EA95F90000112046EFF7879E6B5074F
:1005F50005780EE6601A7BFF7A0779F912081178FB
:100605000EA6071208827FF47E01120935020587BE
:10061500787AE6756200F5637567FF756807756931
:10062500AB85626AF56B7B007A00795912005F7BB6
:10063500FF7A0779F91208117F647E001209357572
:1006450067007568007569597B007A007951120950
:0E065500BB7FD07E071209351209A20205876D
:010663002274
:10095A00C2AD75C804758780759870758921758DC3
:10096A00FD858D8BD28EC2ABD2AFC2A8D288C2CA45
:05097A00D2ACC20A220C
:0300000002071FD5
:0C071F00787FE4F6D8FD7581B302076610
:10035F00E709F608DFFA8046E709F208DFFA803E80
:10036F0088828C83E709F0A3DFFA8032E309F6086D
:10037F00DFFA8078E309F208DFFA807088828C83D5
:10038F00E309F0A3DFFA806489828A83E0A3F60889
:10039F00DFFA805889828A83E0A3F208DFFA804C63
:1003AF0080D280FA80C680D4806980F2803380103A
:1003BF0080A680EA809A80A880DA80E280CA8033A3
:1003CF0089828A83ECFAE493A3C8C582C8CCC5831B
:1003DF00CCF0A3C8C582C8CCC583CCDFE9DEE780EB
:1003EF000D89828A83E493A3F608DFF9ECFAA9F06A
:1003FF00EDFB2289828A83ECFAE0A3C8C582C8CCC0
:10040F00C583CCF0A3C8C582C8CCC583CCDFEADED8
:10041F00E880DB89828A83E493A3F208DFF980CC3A
:10042F0088F0EF60010E4E60C388F0ED2402B40433
:10043F000050B9F582EB2402B4040050AF232345DA
:06044F0082239003AF734D
:10045500BB010689828A83E0225002E722BBFE02A5
:09046500E32289828A83E49322D8
:10046E00BB010CE58229F582E5833AF583E0225043
:10047E0006E92582F8E622BBFE06E92582F8E2228D
:0D048E00E58229F582E5833AF583E49322A7
:10049B00BB010689828A83F0225002F722BBFE0140
:0204AB00F3223A
:1004AD00F8BB010DE58229F582E5833AF583E8F085
:1004BD00225006E92582C8F622BBFE05E92582C831
:0204CD00F22219
:10000300E5732467F8E6057322786430070278679E
:10001300E475F0011204CF0204552000EB7F2ED2C9
:10002300008018EF540F2490D43440D4FF30040BD5
:10003300EF24BFB41A0050032461FFE57460021576
:10004300740577E5777002057630070D7864E475FB
:10005300F0011204CFEF02049B02090E7403D207CE
:100063008003E4C207F5738B648A658966E4F574DB
:10007300F576F577E57460077F2012003E80F5750D
:1000830075FFC201C200C202C203C205C206C20892
:1000930012000CFF700D3007057F0012004FAF7781
:1000A300AE7622B4255FC2D5C20412000CFF24D061
:1000B300B40A00501A75F00A787430D50508B6FFF3
:1000C3000106C6A426F620D5047002D20380D924E3
:1000D300CFB41A00EF5004C2E5D20402024FD2019A
:1000E30080C6D20080C0D20280BCD2D580BAD205ED
:1000F30080B47F2012003E2002077401B5740040D3
:10010300F1120003FF12003E020077D208D20680EC
:1001130095120003FB120003FA120003F94A4B7015
:100123000679207A037BFF20022EE574602A7E0085
:100133008E8275830012046E60060EEE657570F094
:10014300C2D5EBC0E0EAC0E0E9C0E0EE120296D00F
:10015300E0F9D0E0FAD0E0FB120455FF60AAEBC04F
:10016300E0EAC0E0E9C0E012003ED0E02401F9D0AB
:10017300E03400FAD0E0FBE5750460DCD575D98086
:10018300877BFF7A027992D202809C791080027970
:1001930008C206C2088008D2D5790A8004790AC247
:1001A300D5E575047002F575E4FAFDFEFF12000350
:1001B300FC7B08200113120003FD7B1030000A12A0
:1001C3000003FE120003FF7B20EC3382D592D5504F
:1001D30013C3E43000069FFFE49EFEE42001039D69
:1001E300FDE49CFCE4CBF8C201EC700CCFCECDCC8B
:1001F300E824F8F870F38017C3EF33FFEE33FEED16
:1002030033FDEC33FCEB33FB994002FB0FD8E9EBF6
:10021300300105F8D0E0C448B201C0E00AEC4D4E0D
:100223004F78207B0070C2EAB5750040BCC0E01275
:100233000298D0F0D0E0200104C4C0E0C4B201C0F1
:10024300F0120027D0F0D5F0EB0200771204DF01A3
:100253001453018E5800E54C00E14201924F019A7C
:0F02630044019A4900FA4301A0550184460184E1
:100272004501844703405000E92D00ED2E01102B6B
:1002820000F123010E2003292A00A94800000108D9
:100292003F3F3F00790AA2D5200314300509B91067
:1002A200020404B9080104A2D52006025001042068
:1002B20002689202B574005034C0E07F2030031906
:1002C2007F30A20272067205500F1202EFC202C202
:1002D20006C205C2087F30800F300503E9C0E01274
:1002E200003E300503D0E0F9D0E0B574CC300517FC
:1002F2007F30B9100C12003E7F583004077F78809F
:1003020003B9080312003E3002057F2D02003E7F32
:10031200202008F87F2B2006F322920280CF286E3D
:10032200756C6C2900D2011200033001F8C2017809
:100332007430D50108F60200A92D50434958120025
:10034200032403B405004001E490033B9312002F01
:0D035200743A12002FD20375740402018E5C
:10072B00020505E493A3F8E493A34003F68001F2DA
:10073B0008DFF48029E493A3F85407240CC8C333CF
:10074B00C4540F4420C8834004F456800146F6DF9E
:10075B00E4800B010204081020408090084FE47ED7
:10076B00019360BCA3FF543F30E509541FFEE49393
:10077B00A360010ECF54C025E060A840B8E493A35A
:10078B00FAE493A3F8E493A3C8C582C8CAC583CA85
:10079B00F0A3C8C582C8CAC583CADFE9DEE780BE3D
:010881000076
:1004CF00FAE6FB0808E6F925F0F618E6CA3AF6222E
:1004DF00D083D082F8E4937012740193700DA3A3AC
:1004EF0093F8740193F5828883E4737402936860C0
:0604FF00EFA3A3A380DFC0
:10090E00EFB40A07740D120919740A309811A899D8
:10091E00B8130CC2983098FDA899C298B811F63049
:07092E0099FDC299F5992221
:00000001FF
